:020000020000FC
:10000000A2C318C017C016C015C014C013C012C0B8
:1000100011C010C00FC00EC00DC00CC00BC00AC074
:1000200009C008C007C006C005C004C003C002C0A4
:1000300001C000C0EA95F1F708952A985C98299AC2
:1000400008952A985C9A299808952A9A5C98299884
:1000500008952A9A5C9A299A08952A985C98299872
:100060000895EE27E093C500ECE0E093C400E6E0DD
:10007000E093C200E8E1E093C1000895EFE4E0936B
:10008000C600E091C000E6FFFCCFEBE4E093C600C1
:10009000E091C000E6FFFCCFE1E2E093C6000895E6
:1000A0005F9AEF93FF93E4EFF1E0EF93FF93ECECB3
:1000B000F7E03197F1F7FF91EF91319711F000C020
:1000C000F4CFEF91FF915F98EF93FF93E4E6F0E0B8
:1000D000EF93FF93ECECF7E03197F1F7FF91EF919D
:1000E000319711F000C0F4CFEF91FF915F9AEF9339
:1000F000FF93E4EFF1E0EF93FF93ECECF7E031973F
:10010000F1F7FF91EF91319711F000C0F4CFEF912B
:10011000FF91439AEF93FF93E4EFF1E0EF93FF93A6
:10012000ECECF7E03197F1F7FF91EF91319711F097
:1001300000C0F4CFEF91FF914398EF93FF93E4E673
:10014000F0E0EF93FF93ECECF7E03197F1F7FF91DC
:10015000EF91319711F000C0F4CFEF91FF915F98CC
:1001600043980895E0917A00E6FDFCCFE091780095
:10017000F09179000895E091C000E6FF0895CF93D3
:10018000DF9310915004C0E5D4E0C395E991F99153
:10019000DF91CF91113008F408950091C000006400
:1001A0000093C000E093C6001A9511F0F093C600CA
:1001B000CF93DF9310915004112309F11F922F92D6
:1001C0003F924F92C0E5D4E0CD5F199029903990CD
:1001D0004880CA954A923A922A921A92173030F081
:1001E000CA5F19902880CA952A921A921A9509F026
:1001F0001A95109350044F903F902F901F90DF91CD
:10020000CF910895E7E6E0937C00E0917A00E06406
:10021000E0937A00A7DF42E050D00895E6EEE09345
:100220007C00E0917A00E064E0937A009BDFFF932A
:1002300004D0FF9143E041D00895FA3008F001D096
:1002400008954AE028D0439AEF93FF93E8EEF3E055
:10025000EF93FF93ECECF7E03197F1F7FF91EF911B
:10026000319711F000C0F4CFEF91FF9184DFEF934D
:10027000FF93E8EEF3E0EF93FF93ECECF7E03197B8
:10028000F1F7FF91EF91319711F000C0F4CFEF91AA
:10029000FF9159C2089510915004173060F40F93E4
:1002A000042FC0E5D4E0C10FC3950993F9930F91D2
:1002B0001E5F109350045FDF0895109150041730B3
:1002C000D8F4C0E1D4E0C40F08810F1710F00F1B61
:1002D00004C0FF93F01B0F2FFF91013068F0F883EB
:1002E0000F93042FC0E5D4E0C10FC3950993F99390
:1002F0000F911E5F109350043EDF0895109150043B
:100300001630A0F4C0E0D4E0C40FC40FF993E88322
:100310000F93042F005FC0E5D4E0C10FC39509938C
:10032000F993E8830F911D5F1093500424DF089523
:10033000C0E2D4E0E0E1E993E4EDE993E3EAE99394
:10034000E9E8E993E9E7E993EDE6E993E4E6E9937F
:10035000EEE5E993E8E5E993E3E5E993EFE4E99372
:10036000ECE4E993E8E4E993E6E4E993E3E4E99370
:10037000E1E4E993EFE3E993EDE3E993ECE3E99357
:10038000EAE3E993E9E3E993E7E3E993E6E3E99351
:10039000E5E3E993E4E3E993E3E3E9930895EFEF19
:1003A000C0E0D4E0E993C038E8F30895E2E6E093D2
:1003B0007C002B9A5C9AF0E0EBE1EF93FF93EF93D4
:1003C000E5E1EA95F1F7EF910000319729F000C0DF
:1003D00000C000C00000F3CFFF91EF91E0917A00E0
:1003E000E064E0937A00E1E09AD35C982B98BADE5F
:1003F00008955B9A2A9AF0E0EBE1EF93FF93EF9375
:10040000E5E1EA95F1F7EF910000319729F000C09E
:1004100000C000C00000F3CFFF91EF91E0917A009F
:10042000E064E0937A00E1E07AD32A985B989ADE60
:100430000895E1E6E0937C002B9A299AF0E0EBE145
:10044000EF93FF93EF93E5E1EA95F1F7EF91000069
:10045000319729F000C000C000C00000F3CFFF9129
:10046000EF91E0917A00E064E0937A00E1E057D305
:1004700029982B9877DE08955D9A2A9AF0E0EBE1AF
:10048000EF93FF93EF93E5E1EA95F1F7EF91000029
:10049000319729F000C000C000C00000F3CFFF91E9
:1004A000EF91E0917A00E064E0937A00E1E037D3E5
:1004B0002A985D9857DE0895E0E6E0937C005B9A09
:1004C000299AF0E0EBE1EF93FF93EF93E5E1EA95F2
:1004D000F1F7EF910000319729F000C000C000C093
:1004E0000000F3CFFF91EF91E0917A00E064E09398
:1004F0007A00E1E014D329985B9834DE08955D9A80
:100500005C9AF0E0EBE1EF93FF93EF93E5E1EA957E
:10051000F1F7EF910000319729F000C000C000C052
:100520000000F3CFFF91EF91E0917A00E064E09357
:100530007A00E1E0F4D25C985D9814DE0895E12D34
:10054000E40DE0933003E22DE50DE0933103E32D5C
:10055000E60DE0933203E12DE20DE0933303E12D4C
:10056000E60DE0933403E22DE30DE0933503E32D34
:10057000E40DE0933603E42DE50DE0933703E52D1C
:10058000E60DE093480310903303309032031318C4
:1005900008F403C01092440303C0112410924403D2
:1005A0001090360330903103131808F403C01092F2
:1005B000450303C011241092450310904803309066
:1005C0003003131808F403C01092460303C011242B
:1005D000109246031090300330903503131808F43E
:1005E00003C01092470303C01124109247031090D8
:1005F000320330903703131808F403C010924803F5
:1006000003C011241092480310903103309034033A
:10061000131808F403C01092490303C01124109268
:1006200049031090440320904503309046034090C6
:1006300047035090480360904903F1E0812C28144F
:1006400008F402C0F2E0822C381408F402C0F3E08F
:10065000832C481408F402C0F4E0842C581408F4E5
:1006600002C0F5E0852C681408F402C0F6E0862C80
:1006700080924A03F0934B03869480924C03F130AE
:1006800009F40DC0F23009F418C0F33009F423C0A6
:10069000F43009F42EC0F53009F439C046C0F3E057
:1006A000E12DE619E81508F002C0F0E00895E12D0B
:1006B000E419E81508F4F6E00895FFE0E22DE419E6
:1006C000E81508F002C0FCE00895E22DE519E815F0
:1006D00008F4F2E10895FBE1E32DE519E81508F0CF
:1006E00002C0F8E10895E32DE619E81508F4FEE1EB
:1006F0000895F9E0E42DE119E81508F002C0F6E0EC
:100700000895E42DE219E81508F4FCE00895F5E1F8
:10071000E52DE219E81508F002C0F2E10895E52D93
:10072000E319E81508F4F8E10895F1E2E62DE3197C
:10073000E81508F002C0FEE10895E62DE119E8157C
:1007400008F4F0E00895E3E0EEBFE0E0EDBFF894D8
:10075000E0E1E5BF239A539A559A229A549A219A36
:100760003B9A579A519AEE27E5B9E8B9EBB979DC8B
:1007700016DEDEDDE0E4E0937B00EEE4E0937C0057
:10078000E7ECE0937A00EF93E0E0E0935004EF9120
:1007900075DCE8DCEF93FF93E8ECF0E0EF93FF9378
:1007A000ECECF7E03197F1F7FF91EF91319711F011
:1007B00000C0F4CFEF91FF91DEDCEF93FF93E8EC04
:1007C000F0E0EF93FF93ECECF7E03197F1F7FF9156
:1007D000EF91319711F000C0F4CFEF91FF91E7EC6A
:1007E000E0937A00BFDC41E089DDE3E8E0937A0042
:1007F000EF93FF93E1E0F0E0EF93FF93ECECF7E091
:100800003197F1F7FF91EF91319711F000C0F4CFDC
:10081000EF91FF91B0DCF6DCEF93FF93E1E0F0E0C5
:10082000EF93FF93ECECF7E03197F1F7FF91EF9145
:10083000319711F000C0F4CFEF91FF919CDCEEDC1A
:10084000EF93FF93E1E0F0E0EF93FF93ECECF7E040
:100850003197F1F7FF91EF91319711F000C0F4CF8C
:10086000EF91FF9188DC1CDC86DC67D1EF93FF936E
:10087000E4EFF1E0EF93FF93ECECF7E03197F1F761
:10088000FF91EF91319711F000C0F4CFEF91FF91FC
:1008900072DCEF93FF93E4EFF1E0EF93FF93ECEC66
:1008A000F7E03197F1F7FF91EF91319711F000C028
:1008B000F4CFEF91FF915FDCEF93FF93E4EFF1E072
:1008C000EF93FF93ECECF7E03197F1F7FF91EF91A5
:1008D000319711F000C0F4CFEF91FF914CDCEF9312
:1008E000FF93E4EFF1E0EF93FF93ECECF7E0319747
:1008F000F1F7FF91EF91319711F000C0F4CFEF9134
:10090000FF9139DCEF93FF93E8E8F3E1EF93FF9376
:10091000ECECF7E03197F1F7FF91EF91319711F09F
:1009200000C0F4CFEF91FF9101D0FECF3FDDF093F7
:10093000030341E2C2DCEF93FF93E1E0F0E0EF93C9
:10094000FF93ECECF7E03197F1F7FF91EF913197DE
:1009500011F000C0F4CFEF91FF910DDC4ADDF09370
:10096000060344E2AADCEF93FF93E1E0F0E0EF93AB
:10097000FF93ECECF7E03197F1F7FF91EF913197AE
:1009800011F000C0F4CFEF91FF91F5DB52DDF09351
:10099000040342E292DCEF93FF93E1E0F0E0EF9397
:1009A000FF93ECECF7E03197F1F7FF91EF9131977E
:1009B00011F000C0F4CFEF91FF91DDDB5DDDF0932E
:1009C000070345E27ADCEF93FF93E1E0F0E0EF9379
:1009D000FF93ECECF7E03197F1F7FF91EF9131974E
:1009E00011F000C0F4CFEF91FF91C5DB65DDF0930E
:1009F000050343E262DCEF93FF93E1E0F0E0EF9365
:100A0000FF93ECECF7E03197F1F7FF91EF9131971D
:100A100011F000C0F4CFEF91FF91ADDB70DDF093EA
:100A2000080346E24ADCEF93FF93E1E0F0E0EF9346
:100A3000FF93ECECF7E03197F1F7FF91EF913197ED
:100A400011F000C0F4CFEF91FF9195DB1F922F9230
:100A50003F924F925F926F927F928F92109003031A
:100A60002090040330900503409006035090070344
:100A700060900803712C812C281408F0822C271414
:100A800008F4722C381408F0832C371408F4732CF3
:100A9000481408F0842C471408F4742C581408F0F7
:100AA000852C571408F4752C681408F0862C6714EC
:100AB00008F4762C8092090370920A03E82DE71956
:100AC000E03808F408C01694269436944694569458
:100AD000669476948694171827183718471857186D
:100AE0006718871877181092030320920403309236
:100AF0000503409206035092070360920803709228
:100B00000A03809209031BDD8F907F906F905F90A6
:100B10004F903F902F901F9047E2CFDB0895EF93C7
:100B2000EA9521F4EF91000000C0089500C000C0D4
:100B300000C000C000C00000F3CF38DCF093030316
:100B400041E2BBDBEF93FF93E4E6F0E0EF93FF932A
:100B5000ECECF7E03197F1F7FF91EF91319711F05D
:100B600000C0F4CFEF91FF9106DB43DCF093060366
:100B700044E2A3DBEF93FF93E4E6F0E0EF93FF930F
:100B8000ECECF7E03197F1F7FF91EF91319711F02D
:100B900000C0F4CFEF91FF91EEDA4BDCF093040349
:100BA00042E28BDBEF93FF93E4E6F0E0EF93FF93F9
:100BB000ECECF7E03197F1F7FF91EF91319711F0FD
:100BC00000C0F4CFEF91FF91D6DA56DCF093070323
:100BD00045E273DBEF93FF93E4E6F0E0EF93FF93DE
:100BE000ECECF7E03197F1F7FF91EF91319711F0CD
:100BF00000C0F4CFEF91FF91BEDA5EDCF093050305
:100C000043E25BDBEF93FF93E4E6F0E0EF93FF93C7
:100C1000ECECF7E03197F1F7FF91EF91319711F09C
:100C200000C0F4CFEF91FF91A6DA69DCF0930803DE
:100C300046E243DBEF93FF93E4E6F0E0EF93FF93AC
:100C4000ECECF7E03197F1F7FF91EF91319711F06C
:0C0C500000C0F4CFEF91FF918EDA089500
:00000001FF
